:020000040000FA
:020000000528D1
:080008003428831685018601EE
:100010000617861781128111011181138312203076
:10002000A5008B168B17BD01BE01BF01B201B30144
:10003000061F1E20861F26202F2018288B13BD0A7E
:100040003D08183A0319BD018B1708008B13BF0137
:10005000BE0A3E083C3A0319BE018B170800B20BDA
:100060002F28B30B2F280800B0000308B1009D0310
:10007000031965209D1F06169D1B06124E207C202D
:100080002508840000089520A50A2508243A0319AC
:1000900079203108830030080B1109003E08A701C0
:1000A000F63EA70A031850280A3EA703A300270814
:1000B000A2003D08A701F63EA70A03185B280A3EE6
:1000C000A703A1002708A0000800C8309D00BF0AB0
:1000D0003F083C3A031D0800BF01BE0A3E083C3AF7
:1000E000031D0800BE01BD0A3D08183A0319BD01F1
:1000F00008002030A50008002508203A0319051043
:10010000031D05142508213A03198510031D8514C4
:100110002508223A03190511031D05152508233A60
:1001200003198511031D851508000F398604F03861
:04013000860500340C
:02400E00F23F7F
:00000001FF
